:020000040000FA
:020000002528B1
:08000800B529D60000308A0082
:10001000383056028207F1341234F134E834F234C5
:10002000B334F3347234F4342634F434D134F53444
:100030007134F6340934F6349834F7341F34F73415
:100040009F34F8341734F834893483018B018501E7
:100050000730990083161830850070308F00883083
:1000600081000C1083128B12013090000B178B173C
:1000700081214820B321831621309B001C141A08CB
:100080008312C600C700C401C5014708850068285F
:100090004E205A204E205A204E2008000730CA0019
:1000A0004A08083C8500AF2100308500AF21CA0B0B
:1000B000502808000630CA004A03031967284A0876
:1000C0008500AF2100308500AF21CA0B5C280800F5
:1000D000851974288B124410C70A0130C719C7004C
:1000E00047088500B3216828051EB32844187F28D7
:1000F00044140130C8003C30C900FF20682848087B
:10010000031D68288B12441085010130C8000A3095
:10011000C900FF20C50148080319A12845187C2102
:10012000C50105081839183A03198B288B12AF211D
:1001300005081839183A031D9828AF21470885008B
:1001400068288B12C501B1219321850183161830CF
:10015000960083128B15630005081839183A0319A5
:10016000AA28AF2198284708C8003C30C900FF20C2
:1001700085014514451CCF2848088500AF2185011D
:10018000C50149083C3C03197C21480BCF2849088C
:100190000A3C03186E21490BCF28B221D228051A38
:1001A000BA28C4018B1285014418D9289321B121A2
:1001B000FB28C401470846020319EF2883162130A3
:1001C0009B0083124708C60083169A001C15553001
:1001D0009D00AA309D009C149C18EC2883120230CC
:1001E000CA000130D1005130D2000721051EFB2882
:1001F000B121CA0BF12847088500B22168283830A0
:1002000081002430C0002330C1008B16080001306B
:10021000D0004821CD004D0803193F294821CE00C8
:1002200080304D0203193129C0304D02031D1B29B6
:100230004E08CF003C29C1304D02031D262951082C
:10024000D3005208D4004E08D0003C2903104D0DB5
:100250000520C20003144D0D0520C30083160C14A5
:1002600083124F08D5000130A021D50B3329CE0BC6
:10027000312983160C108312051A09294729D00B3E
:10028000422947295308D1005408D20009290800FF
:100290004D21D20A0319D10A080051088A005208D8
:1002A0008200C034233480340834233404342534A9
:1002B000043427341834253404342334043480348B
:1002C0000C342334043425340434273404342534E2
:1002D000043423340434253420340034F630C2008E
:1002E0000930C300643098210800F830C20089301A
:1002F000C3006430982108006E210F30A0216E21C8
:1003000008006E21AD2175210800F130C2001230C5
:10031000C300643098210800F130C2001230C300DD
:10032000FA309821080085216430A0218C21080032
:1003300083160C148312A02183160C10831208005C
:10034000CB00DD30CC00A429A529A629CC0BA329FC
:10035000A929AA29CB0BA12908001E30A0293230D7
:10036000A029B221B321FA30A029F0000308F1003E
:1003700083120B19C0290C18D9290B18E129E62979
:100380000B11383081000130C1020319CB29031849
:10039000E629C002E629C008031DE6292430C00072
:1003A0002330C1004514C90BE6293C30C900C803FD
:1003B000E6290C1042088F0043088E002030850685
:1003C000E6290B108B1183169601831271088300A6
:0603D000F00E700E0900A2
:02400E00C43FAD
:1042000043006F0070007900720069006700680069
:1042100074002000280043002900200032003000F4
:104220003100390020006200790020004D002E008E
:10423000590061006D0061006D006F0074006F0037
:04424000FF00030078
:00000001FF
